S31508003000B8080020D9320008137D00089378000814
S31508003010117D0008A153000855870008000000002C
S31508003020000000000000000000000000C17E00084B
S31508003030EB53000800000000157D0008C37E000859
S31508003040F3320008F3320008F3320008F3320008BE
S31508003050F3320008F3320008F3320008F3320008AE
S31508003060F3320008F3320008F3320008F33200089E
S31508003070F3320008F3320008F3320008B1530008AF
S31508003080F3320008F3320008F3320008F33200087E
S31508003090A5530008F3320008F3320008F33200089B
S315080030A0F3320008F3320008F3320008F33200085E
S315080030B0F33200080000000000000000F3320008A8
S315080030C0F3320008F3320008F3320008F33200083E
S315080030D0F33200083D870008F3320008F33200088F
S315080030E0F3320008F3320008000000000000000078
S315080030F000000000000000000000000000000000C2
S3150800310000000000F332000800000000F332000857
S315080031100000000000000000F3320008F332000847
S31508003120F3320008F3320008F3320008F3320008DD
S31508003130F332000800000000000000000000000054
S31508003140F3320008F3320008F332000800000000EA
S31508003150F3320008F3320008F3320008F3320008AD
S31508003160F3320008F3320008F332000800000000CA
S31508003170F3320008F33200080000000000000000E7
S31508003180F3320008F3320008F332000800F002F8C0
S3150800319000F092F80AA090E8000C82448344AAF151
S315080031A00107DA4501D100F087F8AFF2090EBAE84F
S315080031B00F0013F0010F18BFFB1A43F0010318475D
S315080031C0905C0000B05C0000103A24BF78C878C153
S315080031D0FAD8520724BF30C830C144BF04680C600F
S315080031E0704700000023002400250026103A28BF57
S315080031F078C1FBD8520728BF30C148BF0B6070475B
S315080032006E2900F01583702900F05F84662905F0A1
S315080032107985652905F07685672905F0738561291D
S3150800322005F0728503681B0A28BF41F080016929E9
S3150800323000F0C282642900F0BF82752900F0BC82C2
S315080032406F2900F0ED83782900F02B84E92900F036
S315080032508783E42900F08483F52900F08183EF2928
S3150800326000F0EA83F82900F02A840368DB0928BFFE
S3150800327041F08001632901F07781732901F07C818F
S31508003280E32901F08781F32901F08C81002070473A
S315080032901FB505F032FD01F091FB04000020002166
S315080032A005F09EFC401C60600020002105F082FCB1
S315080032B0E0601FBD10B510BD01F052FB1146FFF7C7
S315080032C0E7FF05F03FFB01F02BFC03B4FFF7F2FF25
S315080032D003BC01F06FFC0000094880470948004715
S315080032E0FEE7FEE7FEE7FEE7FEE7FEE7FEE7FEE7A8
S315080032F0FEE7FEE704480549054A064B7047000005
S31508003300357F00088D310008B8020020B808002073
S31508003310B8040020B804002053EA020C00F06980C3
S315080033202DE9F04B4FF00006002B1FBFB3FA83F5CB
S3150800333003FA05F424FA05F65E4012BF1643B2FAFC
S3150800334082F502FA05F4C5F120051EBF22FA05FC2E
S3150800335044EA0C04203556EA044C4FEA144418BFD4
S31508003360641C4FF000084FF00009904271EB030C03
S3150800337039D3002919BFB1FA81F701FA07F6B0FA6D
S3150800338080F700FA07F6C7F120071EBF20FA07FCE8
S3150800339046EA0C062037B6FBF4FCA7EB0507103FF8
S315080033A007F01F0BCBF120060CFA0BFB2CFA06F6DE
S315080033B044BFB3460026202FA4BF5E464FF0000B3D
S315080033C05BEA060C08BF4FF0010B19EB0B09ABFBC8
S315080033D0027C48EB0608C01B06FB02CC0BFB03CCA1
S315080033E071EB0C01C1E70B46024641464846BDE86B
S315080033F0F08B13B54FF000004FF00001AFF30080DB
S31508003400BDE81C40704700007CB51D4616460C00FA
S31508003410009001D02044401E074B7B442A4669464B
S315080034200190304600F01DFA05461CB10020694699
S3150800343000F02AFA28467CBD750400000FB400B5D2
S315080034408DB010A9099000910B904FF0FF300A90AB
S3150800345000200C90064878440690064878446A4648
S3150800346007900F9909A800F013FC0DB05DF814FB3E
S31508003470570800006F0800002DE9FF5F1D464FF052
S31508003480FF3B91464FF000085F46D5E90146A9691A
S3150800349001987F1C8847296A824688470028F6D102
S315080034A0BAF1FF3F0CD0002E24F4C06419DD600683
S315080034B014D5BAF12B0F09D0BAF12D0F0ED103E0AE
S315080034C0584604B0BDE8F09F44F48064A9690198A1
S315080034D07F1C8847761E8246002E02DDBAF1300F21
S315080034E003D0B9F1000F26D032E0A969761E0198FB
S315080034F07F1C44F400748847002E824605DDBAF125
S31508003500780F06D0BAF1580F03D0B9F1000F10D0D2
S315080035101EE0B9F1000F02D0B9F1100F18D1A96950
S31508003520761E01987F1C24F4007488478246102072
S3150800353002E0082000E00A20814609E0A96908FBA4
S315080035400908761E01987F1C44F400748847824651
S31508003550002E05DD4946504600F086FB0028EDDAC8
S31508003560E96901988847A00502D46FF00100A8E729
S31508003570E00725D1600613D5600502D5C8F100001D
S3150800358000E0404629680A1D2A600968220501D517
S31508003590087015E0220701D5088011E008600FE0E1
S315080035A02868011D29600068210502D580F8008079
S315080035B006E0210702D5A0F8008001E0C0F80080E7
S315080035C038467EE740EA010370B59B072ED14FF0D7
S315080035D00136042A2AD308C810C99D1B9D43121F09
S315080035E015EAC61517D0D8B2E1B2401A50EA0561F5
S315080035F010D198B2A1B2401A50EA05410AD123F077
S315080036007F4024F07F41401A50EA052102D1180E66
S31508003610A0EB146070BDA342DBD018BA21BA884269
S3150800362001D9012070BD4FF0FF3070BD0AB90020E6
S3150800363070BD10F8013B11F8014B63B1A3420AD1E2
S31508003640521E08D010F8013B11F8014B1BB1A342DA
S3150800365001D1521EEDD1181B70BD4FF0000204298E
S31508003660C0F0128010F0030C00F01B80CCF1040CA3
S31508003670BCF1020F18BF00F8012BA8BF20F8022BD7
S31508003680A1EB0C0100F00DB85FEAC17C24BF00F87D
S31508003690012B00F8012B48BF00F8012B70474FF0AB
S315080036A0000200B5134694469646203922BFA0E884
S315080036B00C50A0E80C50B1F12001BFF4F7AF090790
S315080036C028BFA0E80C5048BF0CC05DF804EB890081
S315080036D028BF40F8042B08BF704748BF20F8022BC4
S315080036E011F0804F18BF00F8012B704770477047DC
S315080036F0704770B5044685690068C10601D530264D
S3150800370000E02026C00707D070BDD4E90121304665
S315080037109047206A401C20626D1EF6D570BD70B5B4
S31508003720044685690078C00707D170BDD4E9012130
S3150800373020209047206A401C20626D1EF6D570BD79
S3150800374009684A0501D540B27047C905FCD500B2DB
S31508003750704709684A0501D5C0B27047C905FCD546
S3150800376080B2704770B50C460546012A05D0287800
S31508003770800600D5EA69002302E0012305E05B1C08
S31508003780934202D2E05C0028F9D1A869E618C01A6B
S31508003790A861286A184428622846FFF7AAFF04E0A9
S315080037A0D5E9012114F8010B9047B442F8D328460D
S315080037B0FFF7B5FF70BD00002DE9F041064600246D
S315080037C010687529314616A510D0FFF7B9FF0028ED
S315080037D002DA404213A507E031688A0701D512A527
S315080037E002E0490704D511A5012401E0FFF7B1FF5E
S315080037F000210A2206F1240709E0B0FBF2FCB0FB1F
S31508003800F2F302FB1C00303078541846491C002895
S31508003810F3D123462A463046BDE8F04100F0B6BA51
S31508003820000000002D0000002B0000002000000012
S3150800383011680268006A530501D508700AE0D305C5
S3150800384001D5088006E0130603D5C217C1E90002B0
S3150800385000E008600120704701694A1C0261087887
S31508003860704700B58FB0CDE90131002105910549B2
S315080038707944CDE903101146684600F031F90FB0D6
S3150800388000BD0000E5FFFFFF0A6802F8010B0A60A9
S315080038907047D1E900239A4202D2531C0B6010707C
S315080038A0704700002DE9FF5F15468A460446DFF893
S315080038B0AC80F8440027D8E900103E46CDE9001050
S315080038C010E03AF816106A4602A801F029F8411CD9
S315080038D007D02178890603D5E269391891420DD8AF
S315080038E00744761C2078800602D5E069B84205DDD3
S315080038F0AE42E6DB3AF816000028E2D1A069C01B02
S31508003900A0612046FFF7F5FED8E90010CDE90010C2
S31508003910002017E03AF818106A4602A801F000F8E5
S31508003920B0F1FF3F81460BD000250DF1080B05E0ED
S31508003930D4E901211BF8050090476D1C4D45F7D3C6
S3150800394008F10100B0428046E4DB206A3844206270
S315080039502046FFF7E4FEBDE8FF9F00009E540000E6
S315080039602DE9F0418046D21D22F007020025D2E952
S315080039700002F52915A614D0011E72F1000106DA17
S315080039800023D0EB030063EB020211A608E0D8F887
S3150800399000108B0701D50FA602E0490701D50EA630
S315080039A001251146002408F1240704E000F0A0F9D7
S315080039B030323A55641C50EA0102F7D12B4632469A
S315080039C021464046BDE8F04100F0E0B9000000009D
S315080039D02D0000002B0000002000000030B400215C
S315080039E000F1240408E002F00705D208303542EA5F
S315080039F04372DB086554491C52EA0305F3D104688F
S31508003A00002310A2250708D504F020040C4304D08F
S31508003A10C46901230CA2641EC46130BC00F0B6B9A7
S31508003A2010B5044621461068FFF793FE0246204665
S31508003A30BDE810400023D1E7D21D22F00701D1E9E5
S31508003A400023CBE70000000030000000F0B40D466C
S31508003A500188090502D5214C7C4402E01F4C7C44B0
S31508003A600E34002100F1240608E002F00F071209BF
S31508003A70E75D42EA03721B097754491C52EA0307B9
S31508003A80F3D102780023120704D5702D06D009B1A8
S31508003A90022311342246F0BC00F078B90123103411
S31508003AA0F8E770B504460D4621461068FFF751FE43
S31508003AB0024629462046BDE870400023C6E7D21DC7
S31508003AC022F00703D3E90023C0E70368126843F02E
S31508003AD0200303600823C3610023B7E700530000EF
S31508003AE02DE9F05F894604464FF0000ADFF874B105
S31508003AF0FB44C0F820A02046E1688847002874D017
S31508003B00252806D0D4E901219047206A401C206266
S31508003B10F1E700265F462046E168884720280546E3
S31508003B2007DB312D05D2781910F8200C08B10643A9
S31508003B30F1E7B00701D526F00406C4F81CA0002753
S31508003B40C4F818A02A2D09D0284604F043FE38B335
S31508003B5004EB8708303DC8F8185019E059F8041BDB
S31508003B60204604EB87029161E1688847012F0546E4
S31508003B7018D1E069002820DA26F020061DE0D8F8DA
S31508003B80180000EB800005EB40003038C8F8180034
S31508003B902046E1688847054604F01CFE0028EED159
S31508003BA0012F0AD02E2D08D12046E16888477F1CB0
S31508003BB00546022F46F02006C4DBA069002803DA72
S31508003BC0404246F00106A061F00701D026F0100633
S31508003BD06C2D0BD0682D09D04C2D39D06A2D35D0D7
S31508003BE0742D35D07A2D33D016E038E0E1682F46AB
S31508003BF020468847B842054609D16C2F26D04FF48F
S31508003C008060E168064320468847054604E06C2F35
S31508003C101AD04FF4807006430DB3A5F14100192858
S31508003C2002D8203546F400664A46294620462660CC
S31508003C304E46FFF7E5FA80B101280BD0F61D26F0AF
S31508003C40070000F1080956E74020E4E78020D8E796
S31508003C500020D6E706F104094DE7284652E7206A10
S31508003C60BDE8F09F905200003A2800D2303820F084
S31508003C702002412A01D3A2F13700884201D34FF02E
S31508003C80FF30704702681144137801601846704780
S31508003C90D16005497944516104497944116200218A
S31508003CA01161114600F082BCEDFFFFFFDD00000048
S31508003CB0426842B1016811F8013B23B1521EC0E9BE
S31508003CC00012184670470121C160881E7047426875
S31508003CD05AB1C368016843B983688B4205D0491E47
S31508003CE0521CC0E90012002070474FF0FF307047A1
S31508003CF030B5B0F10A024FEA900E71F100034EEAB0
S31508003D00817EB0EB0E0061EB91014FEA101E4EEA80
S31508003D10017E10EB0E0041EB11114FEA102E4EEA10
S31508003D20016E10EB0E0041EB11214FEA104E4EEAE0
S31508003D30014E10EB0E0041EB1141401841F1000114
S31508003D404FEAD00040EA41704FEAD10110EB8005F6
S31508003D504FEA810444EA907444EB01046D1944EB7C
S31508003D600404521BA3414FF0000348BF0A3200D592
S31508003D7030BD401C41F1000130BD10B5044600F0CD
S31508003D8015FE0068005D00F0010010BD2DE9F04742
S31508003D900D4699469246044600F1240801688806AD
S31508003DA004D5E06921F01001216000E00120A84255
S31508003DB001DD471B00E00027A1697A1902EB09001B
S31508003DC0081AA0612078C00602D42046FFF791FCA5
S31508003DD0002608E0D4E901211AF806009047206A6F
S31508003DE0401C761C20624E45F4DB2078C0060AD5B6
S31508003DF02046FFF77EFC06E0D4E9012130209047F3
S31508003E00206A401C2062381EA7F10107F4DC07E08F
S31508003E10D4E9012118F805009047206A401C206261
S31508003E20281EA5F10105F3DC2046FFF778FC20786B
S31508003E30000602D50220BDE8F0870120FBE770479F
S31508003E402DE9FF4F0C461E464FF0FF378BB0D2E9DF
S31508003E500001DDF860800A908A46C1F30A5505B963
S31508003E603D46002108464FF00000BAF1000F00F465
S31508003E70400005DA00EB80004FF4400101EA5000EB
S31508003E804FEA9059B9F1010F00DDB9460A9850EA90
S31508003E904A000ED044F61050A5F2FF3545432F14BC
S31508003EA0B8F1000F1ED07542291E1EDDC9F10002A9
S31508003EB01CE0B8F1010F4FF0000001D0302103E0FB
S31508003EC0F24305E02154401CB042FBDB3046002299
S31508003ED0002121540B99C1F80880C1E900200FB0D0
S31508003EE0BDE8F08FBD1B6D1CDEE74A4600DA694265
S31508003EF006A800F0A7FD06AB93E8070003AB83E826
S31508003F00070050460A9900F05CFE8DE80700A0F508
S31508003F1000501F3800900398002D09DD42F21F015A
S31508003F204A46084403A90390684601F0BBF808E02E
S31508003F30A0F500504A461F3803A90390684601F0C9
S31508003F40C5F88DE807000004000C03D04FF0FF30D9
S31508003F50410800E01046B8F1000F03D00022009295
S31508003F6015461EE0751E05D4FFF7C2FE30326255AF
S31508003F706D1EF9D5B3460122084302D000227F1CE4
S31508003F8004E02078302801D100227F1E002A0997F4
S31508003F9086D01DE0112D07DAFFF7AAFE30326255EA
S31508003FA06D1C50EA0102F5D1084302D00098C8B149
S31508003FB00EE00021681E05E0235C625C635422540F
S31508003FC0401E491C8142F7DBAB46A81B401E0990E0
S31508003FD0002004F80B000B98099AC0F80880C0E97D
S31508003FE0002B7CE711264FF0000859E72DE9F04F22
S31508003FF088460446D21D22F0070191B0D1E9000196
S31508004000CDE90A0104F0A7FB02460B98C00F01D0C0
S315080040102D2007E02068810701D52B2002E020210A
S3150800402001EAC000032A099001D0072A05DB0346E6
S315080040304146204600F0C6FC0BE12078800601D5F3
S31508004040E06900E00620B8F1650F814606D0B8F1B0
S31508004050660F18D0B8F1670F70D131E00020B9F1BA
S31508004060110F009001DB112301E009F101030AAAEF
S3150800407001A90CA8FFF7E4FEDDE90C70002609F19A
S315080040800105834647E001204B4600904FF0004764
S315080040900AAA01A90CA8FFF7D3FEDDE90DB00C9911
S315080040A05D46002610B909F101000D18B9EB0500A7
S315080040B003D4C0F1FF3609F10105A5EB09002BE091
S315080040C0B9F1010F01DA4FF001090020B9F1110F1A
S315080040D00090484601DD112300E003460AAA01A91B
S315080040E00CA8FFF7ADFEDDE90C704D4600268346A9
S315080040F0207800070AD4AB4500DA5D4601A8012DF1
S3150800410004DD411911F8011C302907D04F4502DAA0
S3150800411017F1040F04DA012082460FE06D1EEEE760
S31508004120002F02DCED1B3E4403E0781CA84200DDAC
S315080041307D1CB81B00F1010A4FF0004720780007E4
S3150800414003D4AA4501DB4FF0FF3A0021B7F1004F2F
S315080041500DF143088DF8431024D002202B23002F9D
S3150800416001DA7F422D230A21021EA0F1010000DC9C
S315080041705FB197FBF1FC97FBF1F201FB1C7C17463C
S315080041800CF1300C08F801CDEEE7A8F10100037038
S315080041902188090501D5452100E06521A0F101081E
S315080041A000F8011C09980FA9A1EB0807FF1D00B12B
S315080041B00120411901EBEA70A1693844081A401E2A
S315080041C0A0612078C00602D42046FFF792FA099823
S315080041D028B1D4E901219047206A401C2062207842
S315080041E0C00622D52046FFF784FA1EE0002E04DB1F
S315080041F0B34502DD01A8805D00E03020D4E9012145
S315080042009047206A401C2062761CAAF101005FEAEA
S31508004210000A0AD100F0D2FBC0680168405CD4E904
S3150800422001219047206A401C2062281EA5F101053D
S31508004230DCDC07E0D4E9012118F8010B9047206A75
S31508004240401C2062381EA7F10107F3DC2046FFF761
S3150800425066FA032011B043E62DE9F04F04460D46F1
S31508004260D21D22F0070089B0D0E9009248461746C9
S31508004270394604F070FA0246F80F01D02D2307E0FC
S315080042802068810701D52B2302E0202101EAC0031B
S315080042908DF820300BB1012000E00020032A824669
S315080042A001D0072A04DB2946204600F08BFB3DE1B6
S315080042B02078800601D40D2500E0E569C7F30A5683
S315080042C00D2D49DA00214FEA175B08464FF000002A
S315080042D0002F00F4400007DA00EB80004FF440019D
S315080042E000EBD07001EA60008115012901DD4FF06D
S315080042F0FF3100224FEA850CBCF1180F06D313468E
S31508004300ACF118004FF08052C24003E04FF480131E
S3150800431023FA0CF30CF10C0CBCF1200F04D3ACF10E
S31508004320200C09FA0CF001E007FA0CF000294FF00E
S31508004330004801DD18B90FE00ED140450CD319EB42
S3150800434002095F4121B9404502D19F4329EA020982
S31508004350BBEB175F00D0761C2088000502D57B488A
S31508004360784402E079487844193808AA302302F8D4
S315080043700A30037C0AF10101002E0AF1020A53549D
S315080043806A4602DC4FF0300101E04FF031014FF090
S3150800439001088DF8001002D0A6F2FF3603E059EAAC
S315080043A0470100D06A4E002D02DC2178090704D5A2
S315080043B04FF002082E218DF80110C44600210BE0AB
S315080043C0C7F303433F01C35C491C6D1E02F808305E
S315080043D0052908F1010801DA002DF1DC00210CE0BD
S315080043E000EB1973491C1B786D1E082902F8083062
S315080043F04FEA091908F1010801DA002DF0DC2178E5
S31508004400890602D514E0A8F10108E04505DD02EBAE
S31508004410080111F8011C3029F5D0B8F1000F07DDA5
S3150800442002EB080111F8011C2E2901D1A8F1010897
S31508004430002D05DD3E2102F808106D1E08F1010861
S31508004440407C002E02F8080008F1010804DA2D2045
S31508004450764202F8080002E02B2002F808000A213A
S315080044604FF47A70864208F101080BDB96FBF0F3ED
S31508004470303302F8083096FBF0F308F1010800FB28
S31508004480136601E0642E0CDB642096FBF0F33033F0
S3150800449002F8083096FBF0F308F1010800FB1366F2
S315080044A001E00A2E06DB96FBF1F0303002F8080030
S315080044B008F1010896FBF1F001FB1060303002F8B4
S315080044C00800A16908F1010808EB050202EB0A00D9
S315080044D0081AA0612078C00602D42046FFF709F919
S315080044E0216A08AE01EB0A00206204E0D4E9012142
S315080044F016F8010B9047BAF1010AF7D22078C006E0
S3150800450002D52046FFF7F5F86E4609E016F8010BC6
S315080045103E280FD0D4E901219047206A401C20622A
S31508004520B8F10108F2D22046FFF7F9F809B00320DE
S31508004530BDE8F08F206A2844206203E0D4E901210F
S31508004540302090476D1EEBD3F8E70000444A000080
S3150800455002FCFFFF10B5436913B1AFF3008001E019
S31508004560FFF700F9012010BD127800F124010A7046
S3150800457000224A700122EDE711684FF0FF32E9E7A1
S3150800458010B5436913B1AFF3008001E0FFF78AF96C
S31508004590012010BD128800F1240182840022C28401
S315080045A00122EDE711684FF0FF32E9E72DE9F34FF5
S315080045B04FF0000A0C4656468DB001200C9001F1CA
S315080045C00C000B9062690B980121904705002DD0CD
S315080045D0252D2CD0216A8847C0B162690B98012124
S315080045E09047216A88470028F7D16269411E0B98CF
S315080045F0904700E0761CA1690D988847216A88478C
S315080046000028F7D1E1690D988847DBE7A1690D987D
S315080046108847A842074601D1761CD3E7E1690D9879
S3150800462088477F1C02D1BAF1000F6FD06BE162692F
S315080046300B9800273D46394690472A2804D16269D7
S315080046400B98012190470125DFF8D08262690B9803
S3150800465001219047A0F130010A290AD24745E5DC35
S3150800466007EB870100EB4107303FDFD445F0100523
S31508004670ECE7E90601D46FF000476C280AD04C280D
S3150800468014D0682815D06A280DD074281CD07A282A
S315080046901AD01DE062690B98012190476C2802D058
S315080046A045F0040514E045F002050DE045F0200547
S315080046B00AE062690B9801219047682802D045F004
S315080046C0080505E045F4006562690B9801219047E5
S315080046D0C4E9015765283DD019DC58287AD00CDC86
S315080046E0452837D004DC252826D041289ED131E03C
S315080046F046282FD0472899D12CE05B2877D0612807
S3150800470028D063287CD0642823D15AE0F6E06F28A5
S3150800471048D008DC66281DD067281BD0692821D018
S315080047206E2816D127E0702845D0732868D07528DA
S3150800473047D078280DD14DE0A1690D9888472528DE
S3150800474005463FF469AFE1690D9888476D1C3FF44B
S315080047506AAFD8E00D9923466A466FF00100AFF3B9
S315080047600080C5E045F0400023464FF00002606037
S31508004770A80736D43EE0E8077FF447AF2068011D56
S3150800478021600068290501D506701BE7290701D5B0
S31508004790068017E7A90703D5F117C0E9006111E7F5
S315080047A006600FE745F0400023464FF008026060B8
S315080047B0A80716D41EE040F60E0125EA010060603F
S315080047C016E045F0400023464FF00A026060A8074D
S315080047D007D40FE045F040006060A80708D52346D7
S315080047E010220D996FF00100AFF3008080E007E01A
S315080047F0102223460D996FF00100FEF73DFE77E083
S315080048004FF0000963284F46C8464B46CB4602D0B0
S315080048105B2806D038E0E80601D40120A06001270D
S3150800482032E06269D4F80CB00B98012190475E28F3
S3150800483007D14FF0010949466269D4F80CB00B98C4
S315080048409047216939B900210A4603AB43F821206C
S31508004850491C0829FADBD8B3216949B308F10108CC
S3150800486062690B98012190475D28F4D1B9F1000FD0
S3150800487009D0002003A951F82020D24341F820206E
S31508004880401C0828F7DB03AB2069002820794FEA8B
S3150800489040701ED05B462246CDF80080CDE90197D0
S315080048A00D9900286FF0010020DAAFF300801FE0B1
S315080048B0C11703AA00EBD1614B1121F01F0102EBCE
S315080048C08302411A13680120884003431360C7E72F
S315080048D019E00D99224600286FF00100009702DAC8
S315080048E0AFF3008004E0AFF3008001E0AFF300808F
S315080048F000280ADA401C06D10C9820B14FF0FF3088
S315080049000FB0BDE8F08F5046FAE7E90701D10AF182
S31508004910010A064400200C9054E60000CCCCCC0CCE
S3150800492070B516460C46054600F040F8036893F83D
S315080049300101012806D0FF2C0FD8185D68B10120A7
S315080049402C7070BDD3F807013246214603F20713CF
S3150800495003442846BDE8704018474FF0FF3070BD45
S31508004960754600F0E3F8AE4605006946534620F062
S315080049700700854618B020B5FEF7BCFCBDE8204008
S315080049804FF000064FF000074FF000084FF0000BFD
S3150800499021F00701AC46ACE8C009ACE8C009ACE8B0
S315080049A0C009ACE8C0098D467047000010B500F094
S315080049B005F8001D10BD00BF2942000000487047D9
S315080049C0740200202DE9F0411F46044603260168BB
S315080049D0072A01F4006004DB08B116A505E016A550
S315080049E003E008B115A500E015A521F01000206028
S315080049F0A069C01EA0610FB1401EA0612046FEF747
S31508004A0078FE4FB1D4E9012138469047206A401C08
S31508004A102062C01C206206E0206AFAE7D4E9012178
S31508004A2015F8010B9047761EF8D22046FEF777FE5A
S31508004A30BDE8F0814E414E006E616E00494E46005B
S31508004A40696E66002DE9F047814616468AB03348F6
S31508004A5078440DC88DE80D0030487844801C03ACB6
S31508004A600DC884E80D0041F69B300844372190FBB9
S31508004A70F1F290FBF1F5A5F1800501FB12041B3C50
S31508004A8002D56442012000E00020DFF890A08046AD
S31508004A900027FA44AAF1BE0A0DE0E00709D032461B
S31508004AA0684607EB47010AEB810100F00FFB8DE82A
S31508004AB0070064107F1C002CEFD1184F7F44AC3FD1
S31508004AC018E0E80714D007EB04100DF1180A90E86F
S31508004AD00E008AE80E00C068F04201D198190890C5
S31508004AE0324606A903A800F0F1FA03AB83E80700EB
S31508004AF06D10641C002DE4D132466946B8F1000FEA
S31508004B0003A802D000F0CEFA01E000F0DFFAC9E906
S31508004B100001C9F808200AB0BDE8F087E4430000A0
S31508004B200446AFF300802046FEF7CFFB00487047E7
S31508004B30540200204FF0013C50F8042B51F8043B76
S31508004B409A4221D1A2EB0C03934313EACC1317D153
S31508004B5050F8042B51F8043B9A4215D1A2EB0C03EA
S31508004B60934313EACC130BD150F8042B51F8043BAA
S31508004B709A4209D1A2EB0C03934313EACC13DBD078
S31508004B804FF00000704700BFD01A01BAB1FA81F1A0
S31508004B9001F0180122FA01F0CB40C1F12001DBB285
S31508004BA0C0B2C01A2CFA01F3D11A914311EAC31103
S31508004BB0E6D1704701491820ABBEFEE72600020081
S31508004BC070475FEA400C08BF91F0000F4FEA8C234C
S31508004BD04FEAC12243EA51514FEA1C5018BF00F56B
S31508004BE0F0404FEA300018BF41F000415FEA6C5CC4
S31508004BF000F02980BCF1FF3F08BF40F080407047B5
S31508004C00130C06BF12044FF0100C4FF0000C130ED5
S31508004C1004BF12020CF1080C130F04BF12010CF1A9
S31508004C20040C930F04BF92000CF1020CD30F04BFBF
S31508004C3052000CF1010C11464FF00002A0F11F00C2
S31508004C40A0EB0C00704711F0004F08BF704731F019
S31508004C5000413FF4D5AF0B0C06BF09044FF0100C0A
S31508004C604FF0000C0B0E04BF09020CF1080C0B0FD9
S31508004C7004BF09010CF1040C8B0F04BF89000CF169
S31508004C80020CCB0F04BF49000CF1010CCCF1200338
S31508004C90A0EB0C0022FA03F302FA0CF241EA030134
S31508004CA000F10100704720F07F4C80EA030023F0F2
S31508004CB07F47ACEB070303F57C5300F0004003F194
S31508004CC0FF032DE980494FEA154B09B44FEA14430F
S31508004CD025EA0B4E24EA03480FF2042606EB1327AF
S31508004CE049083E785FEA320203FB0667C7F5000704
S31508004CF007FB06F64FEA54374FEAD64606F1020690
S31508004D0007FB066CCCF1005C4FEA1C472CEA074C03
S31508004D1007FB06F40CFB06F504EB15464FEA961658
S31508004D2034BF00204FF000404FEAD13706FB07FC9E
S31508004D304FEA1C4C0CFB0BF7D21B03FB0CF761EB81
S31508004D4007010CFB0EF7B0EB074072EB17420CFBA2
S31508004D5008F734BFA2EB0742B2EB074261EB1741F3
S31508004D604FEA0C444FEA910706FB07FC4FEA1C4C36
S31508004D700CFB0BF7B0EBC74072EB573203FB0CF793
S31508004D8034BFA2EBC742B2EBC74261EB57310CFB0B
S31508004D900EF7B0EBC70072EB57720CFB08F734BF7F
S31508004DA0A2EBC702B2EBC70261EB5771039F4FEA4A
S31508004DB0816141EA921104EBCC044FEAD1374FEAFC
S31508004DC0826206FB07FC42EA90124FEA80604FEACD
S31508004DD01C4C0CFB0BF7D21B03FB0CF761EB070112
S31508004DE00CFB0EF7B0EB074072EB17420CFB08F70B
S31508004DF034BFA2EB0742B2EB074261EB17414FEA19
S31508004E008C554FEA910704EB9C2406FB07FC4FEAF6
S31508004E101C4C0CFB0BF7B0EBC74072EB573203FB8D
S31508004E200CF734BFA2EBC742B2EBC74261EB57316E
S31508004E300CFB0EF7B0EBC70072EB57720CFB08F7CA
S31508004E4034BFA2EBC702B2EBC70261EB577115EB91
S31508004E504C254FEA816141EA92114FEA82624FEA94
S31508004E60D13742EA901206FB07FC44F100044FEAE8
S31508004E7080604FEA1C4C0CFB0BF7D21B03FB0CF7AC
S31508004E8061EB07010CFB0EF7B0EB074072EB17421C
S31508004E900CFB08F734BFA2EB0742B2EB074261EB03
S31508004EA0174115EB1C154FEA813141EA92414FEA49
S31508004EB0823242EA90424FEA80304FEA0C7644F159
S31508004EC0000448EA03434EEA0B484FF0000EB2EBE3
S31508004ED0080C71EB030724BF624639464EEB0E0EEB
S31508004EE04FF0000B0018524149414BEB0B0BB2EB4C
S31508004EF0080C71EB03077BF1000B24BF62463946A9
S31508004F004EEB0E0E4FF0000B0018524149414BEB89
S31508004F100B0BB2EB080C71EB03077BF1000B24BFFC
S31508004F20624639464EEB0E0E51EA020718BF46F0A6
S31508004F30010616EB0E7655F1000254F1000103D571
S31508004F40BDE88901BDE80088BDE88901BDE80048DB
S31508004F50B619524141EB0101A3F101037047808064
S31508004F607F7E7D7C7B7A79787776767574737271B5
S31508004F7071706F6E6E6D6C6C6B6A6A69686867666D
S31508004F8066656464636362616160605F5F5E5E5DFF
S31508004F905D5C5C5B5B5A5A59595858575756565573
S31508004FA055555454535352525251515050504F4FD5
S31508004FB04F4E4E4D4D4D4C4C4C4B4B4B4A4A4A4925
S31508004FC04949484848474747474646464545454468
S31508004FD04444444343434342424242414141002BF5
S31508004FE026D4770021D01CB54FEA370703B44FF013
S31508004FF010004FF010014FF000000FBCBDE8104044
S315080050000BF1010BBBF1010F08BF5FEA170722BFBF
S3150800501012F1010211F101014FF0004143F10003C1
S3150800502000F0004043EA00007047F9D35708DAE772
S3150800503046EA064613F1400F4FEA16461FDD13F1FE
S31508005040200FDFBF16430A46002120335B42C8D033
S31508005050C3F1200746EA064602FA07F74FEA16465C
S3150800506046EA0706C3F1200722FA03F201FA07F710
S3150800507021FA03F14FF0000342EA0702B1E746EAD4
S31508005080020646EA06464FEA164646EA0106BCBF47
S3150800509046EA0646360C4FF000034FF000024FF082
S315080050A000019EE72DE9C048934630B491E83800E0
S315080050B007C831EA400C48BF34EA430C03D5FFF76A
S315080050C0F2FDFFF78CFFF0BCBDE800882DE9C0486B
S315080050D0934630B491E8380007C810F0804F08BFEF
S315080050E013F0804F03D100F005F8FFF778FFF0BC06
S315080050F0BDE8008820F07F4780EA030023F07F4C54
S3150800510007EB0C03A3F57C5300F00040A3F1FE0364
S3150800511092F0000F00F0B38095F0000F00F0778052
S315080051202DE901494FEA11404FEA144621EA0048A1
S3150800513000FB06FC24EA064708FB06F607FB08F808
S3150800514000FB07F718EB06484CEB164C4FEA124BD8
S3150800515018EB07484FEA15464CEB174022EA0B4E68
S315080051600BFB06FC25EA06470EFB06F607FB0EFEBA
S315080051700BFB07F71EEB064E4CEB164C4FF00006E2
S315080051801EEB074E4CEB174B18EB0B0840F10000D3
S3150800519018EB0E0B58EB000840F100008F1A4FF081
S315080051A000013CBFC943661B14BFB5EB040C0021C4
S315080051B03CBFC943F61B4FEA17444EEA8E0E27EA50
S315080051C004454FEA1C4704FB07622CEA074C05FB1B
S315080051D007F70CFB05F604FB0CFC16EB074642EB3F
S315080051E0174216EB0C4642EB1C421BEB060658EB25
S315080051F00202414146EA9E0601D5BDE80189B61973
S31508005200524141EB0101A3F10103BDE801894FEACF
S3150800521014454FEA114724EA054621EA074C05FBDF
S3150800522007F406FB07F70CFB06F105FB0CFC11EB74
S31508005230074144EB17444FEA124711EB0C4144EB84
S315080052401C4422EA074C05FB07F206FB07F70CFB92
S3150800525006F605FB0CFC16EB074642EB174216EB67
S315080052600C4642EB1C456A1854F1000148BF7047CA
S31508005270B619524141EB0101A3F10103704795F0BC
S31508005280000F37D04FEA11424FEA144721EA024687
S3150800529024EA074C02FB07F106FB07F70CFB06F4AA
S315080052A002FB0CFC14EB074441EB17414FEA154788
S315080052B014EB0C4441EB1C4125EA074C02FB07F5AD
S315080052C006FB07F70CFB06F602FB0CFC16EB07467B
S315080052D045EB174516EB0C4645EB1C42121951F1E6
S315080052E0000148BF7047B619524141EB0101A3F1CD
S315080052F0010370474FEA14454FEA114724EA054669
S3150800530021EA074C05FB07F106FB07F70CFB06F23B
S315080053104FF0000605FB0CFC12EB074241EB174168
S3150800532012EB0C4251EB1C4148BF7047921841EBF7
S315080053300101A3F10103704710B500F010F8C0F39E
S31508005340401010BD10B50E2000F016F804460F20C8
S3150800535000F012F804F00F0140EA012010BD0B20FE
S3150800536000F00AB810B54FF0FF34FFF7E5FF08B1B3
S31508005370002010BD204610BD1FB54FF47A730122D8
S3150800538003A98DE80E00134602466C21034801F076
S31508005390AFF89DF80C0004B010BD000074000020A2
S315080053A0FEE70000014800F0A7BA00004C00002004
S315080053B0014800F0FBBC00005001002030B590F811
S315080053C0444004F01C050124AC40056C6C6004687C
S315080053D063608368102B036803D099600068C26015
S315080053E030BD9A600068C16030BD704772B6FEE78E
S315080053F0144A117F1448012901D003290FD10368E3
S3150800540023F400730360036843F4006303600368CE
S3150800541023F400630360036843F4007303600229FE
S3150800542001D003290BD1016841F48051016001685C
S3150800543021F480510160016841F480610160002017
S31508005440107770470C00002000200240C10705486D
S3150800545003D0416941F004014161416941F4803159
S31508005460416170470020024008494A69C0B222F4E7
S315080054707E7242EAC0004861486940F0020048610D
S31508005480486940F4803048617047000000200240B7
S31508005490054910B54C6944F001044C610260BFF33C
S315080054A06F8F436010BD000000200240094A10B506
S315080054B05469402344F480245461EFF3108272B691
S315080054C010C910C05B1E13F0FF03F9D182F31088D0
S315080054D010BD00000020024070B5054600F050FFE0
S315080054E00646134C08E0681C06D000F049FF801BEE
S315080054F0A84201D3032070BD2069C003F3D42069F4
S315080055000C4908400CD00C494A6802434A60810F8E
S3150800551001D0A169A161810000D02061012070BD80
S315080055202069C00701D001202061002070BD00005D
S3150800553000200240FAC302000C00002001884088BF
S315080055404AF25A52514040BA4840704710B504468C
S31508005550012020800020A070E0702046FFF7EEFFB3
S31508005560A08010BD70B5114801684068CA4372EA48
S31508005570000215D08BB20C0C0D4A44EA0044090E01
S315080055801380947041EA0021D17090801446B3F5D7
S31508005590006F05D21046FFF7D1FFA188884202D0D6
S315080055A00348FFF7D3FF024870BD000000F8030860
S315080055B04400002070B586B00446FFF7BFFFA08000
S315080055C0A17822880B0CE47842EA0141220A1A43A0
S315080055D0002541EA046440EA020600F0C7FD7F2080
S315080055E0029001200390009504A9684600F0F6FC95
S315080055F0044922463346002000F066FD00F05AFDB5
S3150800560006B070BD00F8030890F82020012A07D0DC
S31508005610022A05D0416A41F480214162012070477F
S31508005620006842690A43426100207047F0B590F865
S3150800563020500468A468012D05D0022D03D0416AC4
S3150800564041F480214DE014F0406F01D1E50045D5C5
S31508005650C4F301640125A5401D608D684FF4C0732D
S315080056609DB1CE6835434E6845EAC605066803EB24
S315080056700417F5514FF4C275076805EB04150E6952
S315080056807E51097D012905D009E00E88CD6845EAD5
S315080056904655EBE701684E5946F480764E51117926
S315080056A0D2F805504FF4C67641EA0521056806EB9F
S315080056B00416A9511178D2F801204FF4C47541EAAD
S315080056C00221026805EB04155151006803EB041129
S315080056D0425842F0010242500020F0BD416A41F4AE
S315080056E0001141620120F0BD10B590F82020012A72
S315080056F007D0022A05D0416A41F48021416201207F
S3150800570010BD0068D0F8002242F00102C0F800225D
S315080057100A7D02F01F0301229A40D0F81C329343F7
S31508005720C0F81C32CB69B3B9D0F80C329343C0F831
S315080057300C328C894B6864F31F434C6900EBC40434
S31508005740C4F840320C890B6864F31F434C6900EBBC
S31508005750C404C4F84432CB69012B16D1D0F80C32F4
S315080057601343C0F80C320C884B6864F31F434C692A
S3150800577000EBC404C4F840320C89CB6864F31F43B9
S315080057804C6900EBC404C4F844328B69002BD0F88A
S3150800579004320FD053EA0203C0F804320B69002B17
S315080057A0D0F8143208D01343C0F81432096A012914
S315080057B004D008E09343EFE79343F5E7D0F81C12CB
S315080057C01143C0F81C12D0F8001221F00101C0F8EC
S315080057D00012002010BD704770B590F82040012CCB
S315080057E005D0022C03D0416A41F4802128E00468E0
S315080057F009B32469A40720D04FF4D874056804EBCC
S3150800580001142D5915F00405956005682D591AD00F
S31508005810ED08556005682C5904F00204D4604FF46D
S31508005820DA74056804EB01142E5906F00F06082EE3
S315080058300CD308250DE0E468DCE7416A41F4001161
S315080058404162012070BD6D0D1560E3E72D5905F025
S315080058500F05156105682D59C5F307259561056876
S315080058602C59240C54614FF4DC72046802EB0112C3
S31508005870A4581C700468A458240A5C700468A458C8
S31508005880240C9C700468A258120EDA704FF4DE726B
S31508005890046802EB0112A4581C710468A458240A6F
S315080058A05C710468A458240C9C710468A258120EF2
S315080058B0DA71006829B1016941F02001016100200F
S315080058C070BDC16841F02001C160F8E702460020BA
S315080058D092F82010012901D002290CD111688A6892
S315080058E0520100D501208A68120100D5401C89683A
S315080058F0C90000D5401C70472DE9F05F05460068D1
S3150800590000244669D0F804908768D0F80CB0D0F81F
S3150800591010A0D0F81880F10748D0F90714D0012153
S315080059208160B80703D5284600F0EBF90CE0780744
S3150800593002D54FF4006407E0380702D54FF48054C7
S3150800594002E0284600F0DCF9F80516D529684FF478
S3150800595080708860B80503D5284600F0D4F90CE0B5
S31508005960780502D544F4005407E0380502D544F416
S31508005970804402E0284600F0C5F9F80316D52968E0
S315080059804FF480308860B80303D5284600F0BDF987
S315080059900CE0780302D544F4004407E0380302D546
S315080059A044F4803402E0284600F0AEF9300707D503
S315080059B05FEACB6004D52968102044F40074C860F7
S315080059C070074FF0080707D55FEA0B7004D52868FB
S315080059D0C760284600F058F9B00706D52868C06899
S315080059E0800702D0284600F051F9700607D55FEA0D
S315080059F0CA6004D52968102044F480640861B0069A
S31508005A0007D55FEA0A7004D528680761284600F0BA
S31508005A1047F9F00606D528680069800702D02846A7
S31508005A2000F03FF9B00308D55FEAC96005D52968D3
S31508005A3010204860284600F035F9F00307D55FEADC
S31508005A40097004D528684760284600F05FF93004D5
S31508005A5046D55FEA497040D5F00504D55FEAC870B7
S31508005A6001D044F00104B00504D55FEA887001D579
S31508005A7044F00204700504D55FEA487001D544F085
S31508005A800404300529D518F0700F26D008F07000E8
S31508005A90402815D006DC102809D020280AD030283E
S31508005AA016D10AE050280ED0602811D10EE044F035
S31508005AB008040DE044F010040AE044F0200407E06E
S31508005AC044F0400404E044F0800401E044F48074A7
S31508005AD02868816921F0700181612968042048607D
S31508005AE0002C05D0686A204368622846FFF773FED3
S31508005AF0BDE8F09F70B5040003D094F8200010B1FB
S31508005B0004E0012070BD204600F082F82068016894
S31508005B1041F00101016000F033FC0546052604E06A
S31508005B2000F02EFC401B0A2811D820684068C007E0
S31508005B30F6D02068016821F00201016000F020FC1F
S31508005B4005460BE000F01CFC401B0A2806D9606AD3
S31508005B5040F40030606284F82060D2E7206840682C
S31508005B608007EFD4207E0128206801683DD021F007
S31508005B7080010160607E01282068016838D021F024
S31508005B8040010160A07E01282068016833D021F019
S31508005B9020010160E07E0128206801682ED041F0CE
S31508005BA010010160207F01282068016829D021F0B2
S31508005BB008010160607F01282068016824D021F06F
S31508005BC004010160D4E902010843D4E9041211432F
S31508005BD008436168491E08432168C861002060625D
S31508005BE0012084F82000002070BD41F08001C0E744
S31508005BF041F04001C5E741F02001CAE721F0100154
S31508005C00CFE741F00801D4E741F00401D9E70000E5
S31508005C1010B586B0044614216846FDF740FD1749BD
S31508005C202068884227D11648816D41F00071816548
S31508005C30816D01F000710591C16C41F00201C164EA
S31508005C40C06C694600F0020005904FF44070009061
S31508005C50022001900020029003200390092004905E
S31508005C60084800F097FA00221146142000F090FD2B
S31508005C70142000F07FFD06B010BD0000006400404F
S31508005C80001002400004004870470000024B034A17
S31508005C900021FFF7A1BD00003400002018020020F3
S31508005CA0704770477047000070B5044690F82000AA
S31508005CB0012804D0606A40F40020606218E00220DF
S31508005CC084F820002068016821F00101016000F0D5
S31508005CD057FB05460EE000BF00F052FB401B0A28A2
S31508005CE008D9606A40F400306062052084F8200014
S31508005CF0012070BD20684068C007EDD1606270BDA4
S31508005D00704770477047704770477047704710B5BF
S31508005D1040B190F825100022022905D00421C1635C
S31508005D2080F82420012010BD01680B6823F00103C8
S31508005D300B6001680B6823F00E030B6090F84410A3
S31508005D40046C01F01C03012101FA03F3636080F877
S31508005D50251080F82420002010BD10B590F82510D5
S31508005D600024022903D00421C16301241AE0016832
S31508005D700A6822F001020A6001680A6822F00E0227
S31508005D800A6090F84410036C01F01C02012101FA24
S31508005D9002F25A6080F82510002180F82410816BE1
S31508005DA001B18847204610BDC06B7047F0B4016C3E
S31508005DB00D6801680C6890F8442002F01C0604225D
S31508005DC002FA06F32B4211D063070FD50B689B0620
S31508005DD003D40B6823F004030B6090F8441001F019
S31508005DE01C018A40016C4A60016B26E0022202FA15
S31508005DF006F72F424FF0000C4FF0010321D0A707FA
S31508005E001FD50C68A40605D40C6824F00A040C6097
S31508005E1080F82530184B0168994290F8441001F033
S31508005E201C0102FA01F202D914490A6002E0124979
S31508005E3080394A6080F824C0C16A00291AD0F0BCAB
S31508005E4008470822B2402A4214D0220712D50A6807
S31508005E5022F00E020A6090F84410026C01F01C0150
S31508005E6003FA01F15160C36380F8253080F824C035
S31508005E70416BE2E7F0BC7047800002400404024030
S31508005E8010B568B12C4C026814232C49A24209D2D9
S31508005E902B4C1444B4FBF3F39B00C0E910130BE03E
S31508005EA0012010BD244C64421444B4FBF3F39B0058
S31508005EB04364214B083B0364022380F825301368AA
S31508005EC047F6F074A3431360D0E902231A43D0E9D6
S31508005ED0043423431A4383691A43C3691A43036A7A
S31508005EE01A4303681C6822431A608268B2F5804F19
S31508005EF019D0036C0F228B4202D151F8A83F02E059
S31508005F000D49A0310B6890F8444004F01C04A240E7
S31508005F1093430B6090F84430426803F01C039A40A0
S31508005F200B681A430A600021C163012280F8252004
S31508005F3080F82410084610BD0804024000000240FC
S31508005F40F8FFFDBF70B5044690F824000025012827
S31508005F500ED0012084F8240094F825600020012E34
S31508005F6008D08021E16384F824000125284670BD05
S31508005F70022070BD022684F82560E0632068066862
S31508005F8026F0010606602046FFF718FA206B00285F
S31508005F902068016802D041F00E0106E021F00401F4
S31508005FA001602068016841F00A0101602068016803
S31508005FB041F001010160D9E770B5044600F0E0F947
S31508005FC00546601C02D004480078044400F0D8F95D
S31508005FD0401BA042FAD370BD000000202DE9F05FF7
S31508005FE0054632488946017801290CD001268046A3
S31508005FF006704CF2503B5846FFF76EFA07004FF012
S31508006000000A03D04EE00220BDE8F09F5146404604
S31508006010C8F804A0264C226892050AD521684905C5
S3150800602005D5216821F480612160032109E00677FE
S3150800603008E02268520504D5216821F480612160B0
S31508006040022101772868012807D04FF0FF31C9F8E7
S31508006050001040F2FA3BAE681DE06868FFF7F6F9F3
S315080060605846FFF739FA0746606920F00400606170
S3150800607016E030466968FFF7F7F94CF25030FFF73B
S315080060802BFA0700606920EA0B00606102D0C9F8A4
S31508006090006005E0761CD5E902010844B042E8D85C
S315080060A0FFF7A6F988F800A03846ADE70C000020EF
S315080060B0002002400348416941F000414161002047
S315080060C070470000002002402DE9FF5F254C064678
S315080060D0904620789A4601280BD0012020704CF271
S315080060E0503B5846FFF7F8F907004FF0000904D06F
S315080060F02AE0022004B0BDE8F09F4846C4F80490A0
S31508006100194D2968490504D5286820F48060286057
S315080061100220207726B1012E09D0022E07D00CE0E6
S31508006120424653460198FFF7B3F9012612E0414665
S315080061300198FFF7BBF9022E0AD05846FFF7CCF9AB
S315080061404FEA0007FFF754F984F800903846D1E77C
S315080061504FF480265846FFF7BFF907466869B043EB
S315080061606861EFE70C000020002002400649002085
S315080061704A69002A07DA054A8A60054A8A6049692F
S31508006180002900DA012070470020024023016745F4
S31508006190AB89EFCD2DE9F04FDFF8AC91002303254D
S315080061A0A9F1040B85B04FF0010C0F2709F1040A79
S315080061B0ABF1040EBFE000BF0CFA03F6324075D00F
S315080061C00C7904F00304012C01D0022C1BD184683D
S315080061D000945C0005FA04F80494009C24EA080478
S315080061E00094D1F80C80049C08FA04F8009C48EA4C
S315080061F00408C0F808804468B4430E79C6F300164C
S315080062009E40264346600C79E443A4070AD0C46836
S315080062104FEA430805FA08F6B4438E6806FA08F604
S315080062202643C6600C7904F00304022C10D1DC085E
S3150800623000EB84040294246A5E074FEAD66807FADC
S3150800624008F6B4430E6906FA08F62643029C266247
S3150800625004684FEA430805FA08F6B4430E7906F0CF
S31508006260030606FA08F6264306604C6814F4403F0F
S3150800627060D0364C266E46F001062666246E23F05C
S31508006280030604F001040094314C34440294A468D3
S315080062909E074FEA167807FA08F6B443B0F1904F0E
S315080062A005D02C4EB04204D1012612E042E0002669
S315080062B00FE0294EB04201D102260AE0274EB0422D
S315080062C001D1032605E0264EB04201D1042600E09E
S315080062D0072606FA08F62643029CA660D9F8006047
S315080062E04C46D1F8048096435FEAC82800D5164381
S315080062F02660DAF800405646D1F8048094435FEAEF
S31508006300882800D514433460DBF800405E46D1F88F
S31508006310048094435FEA883800D514433460DEF875
S3150800632000407646D1F8048094435FEAC83800D521
S31508006330144334605B1C0A6832FA03F47FF43CAFFA
S3150800634005B0BDE8F08F00000804014000100240C7
S31508006350000001400004004800080048000C0048FE
S3150800636000100048426921EA02030A4043EA024152
S31508006370816170470AB18161704781627047000088
S3150800638001488068704700000000002090F841200E
S31508006390202A24D190F84020012A20D0012280F812
S315080063A04020242280F841200268136823F0010364
S315080063B013600268136823F4805313600268136835
S315080063C00B43136001680A6842F001020A60202143
S315080063D080F84110002180F84010084670470220D6
S315080063E0704790F84120202A22D190F84020012AAF
S315080063F01ED0012280F84020242280F8412002681D
S31508006400136823F0010313600268136823F47063AA
S3150800641043EA0121116001680A6842F001020A6034
S31508006420202180F84110002180F840100846704766
S315080064300220704770B5040004D094F84100002586
S3150800644010B106E0012070BD84F84050204600F0E7
S3150800645001F9242084F841002068016821F001012F
S3150800646001606068216820F07060086120688168B2
S3150800647021F400418160E0680128A06830D040F42A
S31508006480044021688860E0680228206841682AD0AC
S3150800649021F40061416020684168144A1143416053
S315080064A02068C16821F40041C160D4E904010843A9
S315080064B0A16940EA01202168C860D4E907010843B8
S315080064C0216808602068016841F00101016065647F
S315080064D0202084F84100256384F84250002070BDCE
S315080064E040F40040CDE741F40061D3E700800002A4
S315080064F02DE9FF4F83B00446DDE9108790F8410087
S31508006500DDF848A09B46202876D15FEA080015D01A
S31508006510A7B194F8400001286ED04FF0010984F81D
S315080065204090FFF72DFF0646012200901923D1035C
S31508006530204601F08FFA002872D103E04FF400706C
S3150800654060646DE0222084F84100402084F842000F
S3150800655000256564C4F8248067856563CDE900A6CF
S31508006560DDE904125B46204601F02AFA10B184F8E8
S31508006570405055E0618D35484FF080774FF00078F0
S31508006580FF2905D9A4F828904A463B46009005E01D
S31508006590618D2185009094F8282043462046049969
S315080065A001F040FA5346002204212046009601F0E5
S315080065B051FAA8BB2068406A616A0870606A401C84
S315080065C06062208D401E81B22185608D401E6085E7
S315080065D0608DE0B1D9B95346002280212046009645
S315080065E001F038FAE0B9608DFF2806D9A4F828909A
S315080065F04A463B46009506E026E0608D20850095D4
S3150800660094F8282043462046049901F00BFA608D39
S315080066100028C7D132465146204601F058FA18B12B
S31508006620012007B0BDE8F08F21682020C8612168E5
S315080066304A68074B1A404A6084F8410084F8425079
S3150800664084F840500020ECE70220EAE700240080A6
S3150800665000E800FE30B59DB00446142117A8FDF7E2
S315080066601EF85C216846FDF71AF817492068884223
S3150800667028D18020002500900D95684600F0F6F890
S3150800668008B1FEF7B3FE114CE06C40F00200E0647E
S31508006690E06C17A900F002001C904FF4C040179058
S315080066A01220CDE9180503201A9004201B900848EB
S315080066B0FFF770FDA06D40F48000A065A06D00F4A2
S315080066C080001C901DB030BD0058004000100240EC
S315080066D000040048024881680278114481607047C6
S315080066E00000002010B50024032000F071F80F20E8
S315080066F000F008F808B1012401E000F025F820466A
S3150800670010BD000070B50E4E05460024307898B1CD
S315080067104FF47A71B1FBF0F00A490968B1FBF0F061
S3150800672000F0C6FD40B9102D06D200222946501E9B
S3150800673000F02EF8756000E00124204670BD0000C8
S31508006740000000202C000020094808B5016E41F021
S3150800675001010166016E01F001010091816D41F0B0
S3150800676080518165806D00F08050009008BD000062
S3150800677000100240002809DB00F01F0201219140A9
S315080067804009800000F1E020C0F8001170470000C1
S31508006790F0B40E4B1B680C46C3F30223C3F107057E
S315080067A0042D00D90425191D072901D2002300E06C
S315080067B0DB1E012606FA05F1491E214099409E4036
S315080067C0761E16403143F0BC01F0DDBF0CED00E04B
S315080067D0064900F0070208684FF6FF03184040EA2A
S315080067E00220034A10430860704700000CED00E0E1
S315080067F00000FA051649B0F5007F0868C0F3412085
S3150800680009D0022805D0086820F4C06040F48060EA
S315080068100860002070470128FBD0086820F4C06093
S3150800682040F4007008600B483222006850430A4A58
S31508006830B0FBF2F0401C00E0401E4A69520501D543
S315080068400028F9D148694005E3D5032070470000C0
S31508006850007000402C00002040420F0002480068EB
S3150800686000F4C06070470000007000402DE9F84F42
S31508006870044600270088A84D3E46000515D5606CDD
S3150800688060B1B0F5000F04D0B0F5400F2BD001274A
S315080068900AE0E86840F48030E86024E00021201D22
S315080068A001F03AFA07001ED03E46206880033AD522
S315080068B0A86D4FF00008C00009D4A86D40F08050BC
S315080068C0A865A86D4FF0010800F080500090DFF829
S315080068D04CA2DAF8001041F48071CAF80010FFF7EC
S315080068E04FFD814610E0D5F88800616C20F4400021
S315080068F00843C5F88800D8E7FFF742FDA0EB090072
S31508006900022801D9032705E0DAF80000C005F3D507
S31508006910002F7DD04FEA0706B8F1000F03D0A86D07
S3150800692020F08050A8652078C00707D0D5F88800E1
S31508006930216A20F003000843C5F8880020788007FC
S3150800694007D5D5F88800616A20F00C000843C5F819
S3150800695088002078400707D5D5F88800A16A20F076
S3150800696030000843C5F888002078800607D5D5F892
S315080069708800E16A20F440600843C5F8880020884A
S31508006980800507D5D5F88800E16B20F44020084338
S31508006990C5F888002088400507D5D5F88800216CF9
S315080069A020F440100843C5F888002078400607D52B
S315080069B0D5F88800216B20F440500843C5F88800B4
S315080069C02078000607D5D5F88800616B20F440408A
S315080069D00843C5F888002088C00507D5D5F888007B
S315080069E0A16B20F440300843C5F8880020684FF0B2
S315080069F0006700034FF0806850D5D5F88800A16C71
S31508006A0020F040600843C5F88800A06CB84200E052
S31508006A1005E03BD1E86840F48010E8603EE0D5F830
S31508006A20900010F4407014D0A16D814211D0D5F8B1
S31508006A309000D5F8901020F4407041F48031C5F8E4
S31508006A409010D5F8901021F48031C5F89010C5F84B
S31508006A509000C00711D0FFF793FC074641F288392A
S31508006A6007E000BFFFF78CFCC11B494501D9032687
S31508006A7052E7D5F890008007F4D5D5F89000A16DB7
S31508006A8020F440700843C5F8900045E7404505D115
S31508006A900121201D01F040F900B106462068400397
S31508006AA017D5D5F88800E16C20F040600843C5F892
S31508006AB08800E06CB84204D1E86840F48010E860C9
S31508006AC007E0404505D10121201D01F025F900B157
S31508006AD006462088400411D5D5F88800216D20F097
S31508006AE040500843C5F88800206DB0F1805F05D195
S31508006AF00221201D01F010F900B106462088000485
S31508006B0006D555F8880F616D20F080400843286047
S31508006B103046BDE8F88F00000010024000700040C3
S31508006B202DE9F0470F4605006BD0494E306800F056
S31508006B300700B84209D2306820F0070038433060B1
S31508006B40306800F00700B8425BD12878414C8007CE
S31508006B500AD5A868A16801F0F001884204D9A1689D
S31508006B6021F0F0010143A1602878C0072CD068689D
S31508006B70032811D0022812D0216898B149050029A6
S31508006B803FDAA16821F003010143A160FFF7F8FB92
S31508006B90804641F2883910E021688901EFE72168CB
S31508006BA08903ECE78907EAE7FFF7EAFBA0EB0801A8
S31508006BB0494502D90320BDE8F087A068696800F056
S31508006BC00C00B0EB810FEFD1287880070AD5A868AA
S31508006BD0A16801F0F001884204D2A16821F0F00111
S31508006BE00143A160306800F00700B8420BD930684D
S31508006BF020F0070038433060306800F00700B842DC
S31508006C0001D00120D7E72878400705D5A068E968AC
S31508006C1020F4E0600843A0602878000706D5A0683D
S31508006C20296920F4605040EAC100A06000F03EF8EF
S31508006C30A168094AC1F30311515C01F01F01C8405C
S31508006C400649086006480068BDE8F047FFF75ABDE0
S31508006C5000200240001002400C8D00082C00002085
S31508006C60040000200548064900688968054AC1F3FA
S31508006C700221515C01F01F01C84070472C0000201A
S31508006C80001002404C8D00080548064900688968CE
S31508006C90054AC1F3C221515C01F01F01C840704783
S31508006CA02C000020001002404C8D000870B52449C5
S31508006CB0002318468A68CC6812F00C0204F0030612
S31508006CC0204C214D09D00C2A05D0042A32D0082A96
S31508006CD000D1284670BD012E10D10B681B0704D4BD
S31508006CE0D1F89430C3F3032302E00B68C3F303130C
S31508006CF0164E56F82330DAB10C2AEBD1C86800F0E4
S31508006D000300022818D0032818D01846CA68CB688A
S31508006D10C2F30212C3F306234343521CB3FBF2F237
S31508006D20C868C0F34160401C4000B2FBF0F070BD7B
S31508006D30184670BD204670BD2046E7E72846E5E7B9
S31508006D40001002400024F40000366E011C8D000875
S31508006D502DE9F84304006FD0FA4DA86800F00C0638
S31508006D60E86800F003072078C00664D576B10C2ED3
S31508006D7001D1012F0AD0A069002828687AD040F0EE
S31508006D8001002860FFF7FCFA80465DE02868800766
S31508006D9002D5A0690028DED0216A2868000703D535
S31508006DA0286800F0F00004E0D5F89400F02202EA22
S31508006DB01010814216D9084601F044F800283BD144
S31508006DC0286840F0080028602868216A20F0F0004A
S31508006DD0084328606868E16920F47F4040EA01209A
S31508006DE0686016E0286840F0080028602868216A6C
S31508006DF020F0F000084328606868E16920F47F40C5
S31508006E0040EA0120686026B9206A01F01BF80028CC
S31508006E10D5D1FFF74BFFA968CB4AC1F30311515CE3
S31508006E2001F01F01C840C9490860C9480068FFF752
S31508006E3069FC00287ED12EE0CAE000BFFFF7A0FA61
S31508006E40A0EB0800022876D828688007F6D52868B7
S31508006E5040F0080028602868216A20F0F0000843FE
S31508006E6028606868E16920F47F4040EA012068608C
S31508006E7011E0FFE720F001002860FFF781FA80465D
S31508006E8006E000BFFFF77CFAA0EB08000228DAD874
S31508006E9028688007F6D42078C00740D0082E18D076
S31508006EA00C2E01D1032F14D06068B0F5803F17D09F
S31508006EB0B0F5A02F286817D020F4803028602868FD
S31508006EC020F4802028606068E0B1FFF759FA804610
S31508006ED014E02868800322D56068002878D01EE070
S31508006EE0286840F48030EDE740F480202860F7E712
S31508006EF0FFF746FAA0EB08006428A4D828688003A0
S31508006F00F6D50CE0FFF73CFA804605E0FFF738FABD
S31508006F10A0EB0800642896D828688003F6D4207861
S31508006F2080073BD5042E11D00C2E01D1022F0DD08F
S31508006F30E06801E0AAE1FFE0002828681ED040F4D6
S31508006F4080702860FFF71CFA07460CE028684005A1
S31508006F500CD5E0680028C1D008E000BFFFF710FA9A
S31508006F60C01B022893D828684005F7D56868217C95
S31508006F7020F0F85040EA016068600FE020F4807065
S31508006F802860FFF7FDF9074605E000BFFFF7F8F9A7
S31508006F90C01B0228B1D828684005F7D42078000716
S31508006FA029D560690028D5F8940012D040F0010070
S31508006FB0C5F89400FFF7E4F9074604E0FFF7E0F99F
S31508006FC0C01B022899D8D5F894008007F6D512E098
S31508006FD02BE120F00100C5F89400FFF7D1F9074628
S31508006FE005E000BFFFF7CCF9C01B022885D8D5F805
S31508006FF094008007F6D42078400766D5A86D002748
S31508007000C00008D4A86D40F08050A865A86D012777
S3150800701000F0805000904F480168C90512D40168F5
S31508007020814641F480710160FFF7AAF9804605E0C0
S31508007030FFF7A6F9A0EB080002287DD8D9F80000CA
S31508007040C005F5D5A068012816D00528D5F8900002
S3150800705017D020F00100C5F89000D5F8900020F070
S31508007060040000BFC5F89000A06841F28839C0B195
S31508007070FFF786F980460FE0D5F8900040F001004A
S31508007080F0E740F00400C5F89000F5E7FFF778F957
S31508007090A0EB080149454FD8D5F890008007F5D5EB
S315080070A00EE0FFF76DF9804606E000BFFFF768F9C6
S315080070B0A0EB080149453FD8D5F890008007F5D4DC
S315080070C01FB1A86D20F08050A8652078800628D5C5
S315080070D0606A0028D5F8980012D040F00100C5F87B
S315080070E09800FFF74DF9074605E000BFFFF748F996
S315080070F0C01B022820D8D5F898008007F6D510E0DE
S3150800710020F00100C5F89800FFF73AF9074604E0B1
S31508007110FFF736F9C01B02280ED8D5F89800800765
S31508007120F6D4A06AF0B3022816D00C2E7DD02868B3
S3150800713020F08070286000E0A7E0FFF721F90446F8
S31508007140A6E00000001002400C8D00082C0000206C
S315080071500400002000700040E868E26A00F00301BD
S31508007160914228D1216B00F0700209011039914231
S3150800717021D1626B00F4FE41B1EB022F1BD194F8CA
S31508007180382000F07841B1EBC26F14D1A18F00F41A
S31508007190C00249084905A1F5001191420BD194F89E
S315080071A0401000E06AE04908490600F0C060A1F115
S315080071B0007181424BD00C2E73D02868400170D4E0
S315080071C0286820F080702860FFF7DAF8064604E0A1
S315080071D0FFF7D6F8801B022857D828688001F7D40D
S315080071E0F4E90B016FF00F0202EB01110843218A43
S315080071F05204490802EB4151A26841EA02210843B8
S31508007200217D4FF07E42490802EB41610843217B0C
S3150800721040EAC160E968244A11400843E8602868E2
S3150800722040F080702860E86800E03AE040F080703E
S31508007230E860FFF7A5F8044605E000BFFFF7A0F8E9
S31508007240001B022821D828688001F7D527E028687E
S31508007250800124D4286840F080702860E86840F0EF
S315080072608070E860FFF78CF8044604E0FFF788F8BA
S31508007270001B022809D828688001F7D50FE000BF4F
S31508007280FFF77EF8001B022802D90320BDE8F88321
S3150800729028688001F4D4E86804490840E8600020BA
S315080072A0F4E70120F2E700008C809D01FCFFEEFE6A
S315080072B010B5401EB0F1807F01D3012010BD4FF0FC
S315080072C0E02460610F21601701F05DFA0020A061DB
S315080072D007202061002010BD7047704770B504462E
S315080072E0C06FD4F88060216889684FF010050906D8
S315080072F018D5212816D12068083050E8001F21F03B
S31508007300800140E80012002AF5D1206F38B1FEF757
S31508007310FEFC20B1206FFEF747FD202821D020462D
S3150800732001F065F820688068400618D5222E16D127
S315080073302068083050E8001F21F0400140E800129C
S31508007340002AF5D1606F38B1FEF7E1FC20B1606F15
S31508007350FEF72AFD202804D0204601F022F8002056
S3150800736070BDC4F88450032070BD000010B50446F3
S3150800737000680A49884210D12046FFF7AFFF08493E
S315080073800020087020210748FCF767F92046BDE869
S3150800739010402022034900F0FFB910BD0038014013
S315080073A03C000020340200202DE9F0410268044622
S315080073B0D0691168936840F60F0528424FF000051A
S315080073C04FF0020605D187067ED58F067CD5A16EBD
S315080073D033E1DFF894C203F0010701EA0C0C57EA1F
S315080073E00C0C71D05FEAC07C0CD05FEAC15C09D591
S315080073F04FF0010CC2F820C0D4F8842042F00102F4
S31508007400C4F88420820709D5DA0707D022681662ED
S31508007410D4F8842042F00402C4F8842042070AD52E
S31508007420DA0708D0236804221A62D4F8842042F0C6
S315080074300202C4F8842002070CD501F020023A4360
S3150800744008D0236808221A62D4F8842042F0080279
S31508007450C4F8842002050BD54A0109D523684FF4E0
S3150800746000621A62D4F8842042F02002C4F884200C
S31508007470D4F88420002A36D0800605D5880603D598
S31508007480A16E09B120468847D4F884002168896826
S31508007490490602D410F0280F27D0204600F081FFB5
S315080074A02068806840061BD52068083050E8001F11
S315080074B021F0400140E80012002AF5D1606F78B14A
S315080074C06A498163606F00E015E0FEF746FC002814
S315080074D009D0606F816B00E02046BDE8F04108479F
S315080074E02046FFF743FFBDE8F0812046FFF73EFF41
S315080074F0C4F88450F7E7D4F860C02027BCF1010F20
S315080075007ED15FEAC06C7BD55FEAC16C78D5102066
S3150800751010622068806840064FD5616F0A68506817
S315080075200004000C3DD0B4F85830834239D9A4F889
S315080075305A000868006880062BD4206850E8001FA7
S3150800754021F4807140E80012002AF6D1206808303C
S3150800755050E8001F21F0010140E80012002AF5D189
S315080075602068083050E8001F21F0400140E800126A
S31508007570002AF5D1C4F880702566206850E8001FF7
S3150800758021F0100140E80012002AF6D1606FFEF7DC
S31508007590BEFB6666B4F85800B4F85A10401A81B2B1
S315080075A007E0B4F8581081429DD1106880069AD534
S315080075B066662046FFF790FE95E7B4F85800B4F8DB
S315080075C05A10401A81B2B4F85A0000288BD0002904
S315080075D089D0226852E8000F20F4907042E8000330
S315080075E0002BF6D12068083050E8002F22F001025F
S315080075F040E80023002BF5D1C4F88070256600E02A
S315080076000AE0A566226852E8000F20F0100042E85A
S315080076100003002BF6D1CBE7C60209D55B0207D5D6
S315080076204FF4801010622046BDE8F041FFF755BEC2
S31508007630020606D50A0604D5E16E00297FF44CAF8A
S3150800764051E74006B8D54806B6D52046026852E83E
S31508007650001F21F0400142E80013002BF6D1C7674E
S31508007660C56600F015F93EE720010004858200088A
S3150800767010B5040002D0E06F10B107E0012010BD7C
S31508007680002084F87800204600F026F82420E067D9
S315080076902068016821F001010160606A10B1204686
S315080076A000F050FC204600F0AFFE0128E7D0206825
S315080076B0416821F4904141602068816821F02A01DF
S315080076C081602068016841F0010101602046BDE83B
S315080076D0104000F09BBC0000F0B59DB00646142192
S315080076E017A8FBF7DCFF5C216846FBF7D8FF26499D
S315080076F03068884245D101240025684608950094DB
S31508007700FFF7B4F808B1FDF771FE2048016E41F4A1
S3150800771080410166016E01F480411C91C16C41F003
S315080077200101C164C06C022700F001001C904FF4EF
S31508007730C060CDE917070320CDE9194007201B9043
S3150800774017A94FF09040FEF725FD124C104820600F
S31508007750C4E901758020C4E903506561A561E56146
S3150800776020462562FEF78CFB08B1FDF73FFE7467DD
S31508007770002211462520A662FFF70AF82520FEF703
S31508007780F9FF1DB0F0BD00000038014000100240AE
S31508007790580002405001002030B4D0F88030202B29
S315080077A002D0022030BC7047A9B1A2B100230366FB
S315080077B00A4C0368A3420BD05B681B0208D5046811
S315080077C054E8003F43F0806344E80035002DF6D1C5
S315080077D030BC00F019BF0120E4E70000008000403B
S315080077E0704770472DE9F84F0446C06F984615460E
S315080077F00E46202802D00220BDE8F88F86B37DB356
S315080078000020C4F884004FF02109C4F87C90FEF7E4
S31508007810B7FDA4F850508246A4F85250A068B0F5B7
S31508007820805F01D1206910B13546002600E00025A9
S315080078305FF02007B4F8520053464FF00002CDF827
S315080078400080D0B18021204600F02EFFD0B94DB17E
S3150800785015F8010B21688862E16F39EA010006D044
S315080078600120C9E736F8020BC0F30800F2E7B4F8BE
S315080078705200401EA4F85200DCE74021204600F0E2
S3150800788013FF10B1E7670320B6E7E7670020B3E701
S315080078907047FEE701688A69D243920701D400223D
S315080078A08A6200688169C943C90703D0816941F0C2
S315080078B001018161704700002DE9F0470446006820
S315080078C088460026816935461746C9064FF02009BD
S315080078D03FD51021C1612FE0B8F1FF3F2CD0FEF74C
S315080078E04FFDC11B414502D8B8F1000F24D12068CD
S315080078F0416894F8422001F480418369DB431B0404
S3150800790015D4B1F5804F12D0202A10D0416841F421
S3150800791080414160FEF734FD074608E0FEF730FD7A
S31508007920C01B192803D945F02005012604E0206864
S315080079308069C0438006F1D420688069C0F340108E
S315080079403043C9D016B92168C1F81C9045F0040522
S31508007950012621688869C20505D54FF4807245F06D
S315080079600105CA610126410509D522684FF48061DF
S3150800797045F00805D1610126800502D40AE0800594
S3150800798007D521684FF4007045F00205C861012645
S3150800799000E086B12046FFF77DFF54F8241B4868AF
S315080079A0064A10404860206A2843206284F81D90E1
S315080079B00020A07720773046BDE8F08700E800FE73
S315080079C02DE9F84304461646DDE908971448984613
S315080079D0DAB200900023204600F024F83A464946D9
S315080079E0204600F09FF8B8B9F5B2B8F1010F08D0F3
S315080079F02168300A88623A464946204600F092F8DD
S31508007A0050B9206885624B460022402120460097DF
S31508007A1000F020F8002800D00120BDE8F883000017
S31508007A200020008010B5C1F3090141EA024102684D
S31508007A30029C19432143506821F000414FF48063AA
S31508007A4003EA5453024C234398430843506010BD3D
S31508007A50FF63FF032DE9F0411D4617460E4604460F
S31508007A60DDF8188027E0424629462046FFF724FF1E
S31508007A7010B10120BDE8F081681C1CD0FEF780FC1F
S31508007A80A0EB0800A84200D8ADB92068806936EA9C
S31508007A9000000ED00020B8420DD154F8440F40F033
S31508007AA0200044F80409202060700020A07020708F
S31508007AB0DFE70120EFE72068806936EA000004D096
S31508007AC00020B842CFD00020D4E70120F9E770B5EE
S31508007AD016460D4604461EE0324629462046FFF75E
S31508007AE0EBFE08B1012070BDFEF74AFC801BA842D8
S31508007AF000D885B920688069C04380060BD554F83C
S31508007B00440F40F0200044F804092020607000204B
S31508007B10A0702070E6E720688069C0438006DBD441
S31508007B20002070BD70B516460D46044620E0324664
S31508007B3029462046FFF7C0FE08B1012070BD681C23
S31508007B4016D0FEF71DFC801BA84200D885B9206810
S31508007B508069C04380070BD554F8440F40F02000D5
S31508007B6044F80409202060700020A0702070E4E723
S31508007B7020688069C0438007D9D4002070BD000002
S31508007B800F4810B50D4901601421416000214FF4DA
S31508007B9080328160C0E90312416101760122427692
S31508007BA08176C27601774177FDF7A4FF002803D0D6
S31508007BB0BDE81040FDF71ABC10BD00000064004087
S31508007BC04C000020094808B5816C41F00101816428
S31508007BD0806C002200F00100009011460F20FEF78D
S31508007BE0D7FDBDE808400F20FEF7C4BD00100240CF
S31508007BF0F0B587B014216846FBF751FD1D48C16CE6
S31508007C0041F08001C164C16C01F080010591C16C2D
S31508007C1041F00201C164C16C01F002010591C16C19
S31508007C2041F00101C164C06C012200F00100D403D7
S31508007C304FF09046059021463046FEF79BFB0E4FC7
S31508007C40012238213846FEF795FB009401240025C9
S31508007C50694630460194CDE90245FEF79BFA38207D
S31508007C60CDE9000469463846CDE90245FEF792FAA1
S31508007C7007B0F0BD0010024000040048134810B5D4
S31508007C80114901601249416000210122C0E902122E
S31508007C90016141618161C1610162FEF7CBFB08B1F7
S31508007CA0FDF7A4FB00210948FEF770FB08B1FDF7B4
S31508007CB09DFB00210548FEF794FB002803D0BDE88C
S31508007CC01040FDF793BB10BD00580040740000201B
S31508007CD0E49CD1100D4810B50B4901604FF4E13111
S31508007CE04160002181600C22C160C0E904128161F3
S31508007CF0C16101624162FFF7BBFC002803D0BDE801
S31508007D001040FDF773BB10BD00380140C8000020C5
S31508007D10FEE7FEE7704700002DE9F041444C0546B2
S31508007D208846E0680026810728680DD0E16801F0DA
S31508007D300301814216D1A8B1E0686968C0F3021050
S31508007D40401C88420ED120E0012804D0022805D024
S31508007D50032807D108E02168890701E02168490559
S31508007D60002907DB01265FE02168890302D4216820
S31508007D704903F5E7E1686A686FF00F0321F07301BC
S31508007D8003EB021211430143E160206820F0806092
S31508007D902060FEF7F5FA074605E000BFFEF7F0FAA1
S31508007DA0C01B022837D820680001F7D4B8F1000FA5
S31508007DB018D0B8F1010F1DD0287D4FF07E4140083C
S31508007DC001EB4060A96840EA01202169194A11407F
S31508007DD008432061206840F080602060FEF7D0FAF2
S31508007DE007461AE0A868297B000240EAC1602169B3
S31508007DF0114AECE7288A1149400801EB4050A96866
S31508007E0040EA012021690E4AE1E700BFFEF7B8FA09
S31508007E10C01B022801D9032606E020680001F5D513
S31508007E202069A969084320613046BDE8F081000051
S31508007E3000100240FF80FFF9FF80FF070000E0FF07
S31508007E40FF809FFFF8B51C4D06460024A86DC000AC
S31508007E5002D5FEF703FD0DE0A86D40F08050A86539
S31508007E60A86D00F080500090FEF7F8FCA96D21F08F
S31508007E708051A965B0F5007F04D0802E07D94FF050
S31508007E8003040AE0802E08D9A02E01D804E001D107
S31508007E90022402E0702E00D101240848016821F06E
S31508007EA0070121430160006800F00700A04201D0E5
S31508007EB00120F8BD0020F8BD001002400020024055
S31508007EC07047FEF707BC10B596B044216846FBF725
S31508007ED0E6FB142111A8FBF7E2FB4FF40070FEF74E
S31508007EE089FC08B172B6FEE701200324009000045D
S31508007EF0019002201421CDE90A04CDE90C4107219D
S31508007F00CDE90E1010906846FEF722FF08B172B64A
S31508007F10FEE70F20CDE91104002013901490159068
S31508007F20042111A8FEF7FCFD002801D072B6FEE771
S31508007F3016B010BD0248016841F47001016070472F
S31508007F4088ED00E090F82410090706D501684A680C
S31508007F50436B22F400421A434A6090F82410C9077A
S31508007F6006D001684A68836A22F400321A434A60D6
S31508007F7090F82410890706D501684A68C36A22F46E
S31508007F8080321A434A6090F82410490706D50168DA
S31508007F904A68036B22F480221A434A6090F8241038
S31508007FA0C90606D501688A68836B22F480521A438B
S31508007FB08A6090F82410890606D501688A68C36B1A
S31508007FC022F400521A438A6090F82410490611D503
S31508007FD001684A68036C22F480121A434A60016CED
S31508007FE0B1F5801F06D101684A68436C22F4C002C5
S31508007FF01A434A6090F82410090606D501684A68AB
S31508008000806C22F4002202434A6070472DE9F84347
S3150800801000260446C0F88460FEF7B2F98046206858
S3150800802000684FF0200500076FF07E4712D54346DB
S31508008030002229042046009700F036FB50B121683B
S3150800804051E8000F20F0800041E80002002AF6D12E
S31508008050E56721E020680068400722D543460022EC
S315080080604FF480012046009700F01EFBC8B1216836
S3150800807051E8000F20F4907041E80002002AF6D17A
S315080080802068083050E8001F21F0010140E800127E
S31508008090002AF5D1C4F8805084F878600320BDE83A
S315080080A0F883E567C4F8805044F8606F6660267602
S315080080B00020F4E738B5054600206854052235A1A6
S315080080C02846FBF77FFA354C98B1082234A1284692
S315080080D0FBF778FA002827D0062234A12846FBF7B2
S315080080E071FA00283DD02946BDE8384031A000F095
S315080080F05BBB6A4635A1681DFBF7A0F901282BD1A1
S31508008100FDF730FA606000889DF80010884209D0B3
S315080081100A4601462EA000F047FB60689DF800104D
S31508008120018017E033A019E06A4628A105F1080086
S31508008130FBF784F901280FD19DF80010617034A06F
S3150800814000F032FBFDF70EFA6060C27861788A4269
S3150800815003D0C170FDF72EFA38BD34A000F024FB19
S3150800816038BD6A4619A1A81DFBF768F90128F7D199
S315080081709DF80010A17035A000F016FBFDF7F2F986
S3150800818060608278A1788A4201D08170E2E735A0E2
S31508008190E4E7000053455449440000003C00002031
S315080081A0534554444542554700000000534554443E
S315080081B049520000556E6B6E6F776E20636F6D6D5A
S315080081C0616E643A2025730A0000000025780000D5
S315080081D043757272656E742049443A2030782530AA
S315080081E032582C204E65772049443A20307825307D
S315080081F032580A0043414E20494420756E6368612F
S315080082006E6765643A203078253032580A000000D7
S31508008210536574206465627567206C6576656C3A8B
S31508008220203078253032580A00000000446562750F
S3150800823067206C6576656C20756E6368616E676528
S31508008240643A203078253032580A00005365742085
S31508008250646972656374696F6E3A203078253032C6
S31508008260580A0000446972656374696F6E20756EFA
S315080082706368616E6765643A203078253032580A3B
S315080082800000000010B5806AFFF770F810BD70B5E1
S31508008290846AE06FD4F8805021688968090604D595
S315080082A0212802D1204600F0A2F8206880684006FE
S315080082B004D5222D02D1204600F073F8D4F88400A4
S315080082C040F01000C4F884002046FFF74FF870BD50
S315080082D010B50146806A0A68126892062BD40268AD
S315080082E052E8003F23F4807342E80034002CF6D1AC
S315080082F00268083252E8003F23F0010342E80034DE
S31508008300002CF5D10268083252E8003F23F04003FA
S3150800831042E80034002CF5D12022C0F88020026EF5
S31508008320012A08D1036853E8002F22F0100243E817
S315080083300024002CF6D100224266026E012A02D0E1
S31508008340FFF74EFA10BD09684968B0F8582089B297
S315080083508A4201D9A0F85A10B0F85A10511A89B2AF
S31508008360FEF7BAFF10BD10B50246806A01214166C4
S31508008370016E012902D0FFF734FA10BDB0F8581083
S315080083804B08A0F85A301268526892B2914201D34B
S31508008390A0F85A20B0F85A20891A89B2FEF79CFF2D
S315080083A010BD016851E8002F22F4907241E80023BD
S315080083B0002BF6D10168083151E8002F22F001029E
S315080083C041E80023002BF5D1016E012908D1026886
S315080083D052E8001F21F0100142E80013002BF6D1E5
S315080083E02021C0F880100021016681667047026866
S315080083F052E8001F21F0C00142E80013002BF6D115
S315080084002021C167704700002DE9F0410446016844
S3150800841080682269E3691043626900251A4310439C
S31508008420714F0A68714B1A4002430A602068416816
S31508008430E26821F44051114341602168A069B942BC
S3150800844001D0226A10438A6822F4306202438A60A5
S315080084506749236867488B420DD1D0F8880010F029
S31508008460030006D0012847D0022843D0032830D17C
S3150800847044E001212EE060498B420BD1D0F88800F8
S3150800848010F00C0034D0042836D0082832D00C2836
S315080084901FD133E059498B420BD1D0F8880010F030
S315080084A0300025D0102827D0202823D0302810D1F6
S315080084B024E0BB420DD1D0F8880010F4406017D0F4
S315080084C0B0F5806F18D0B0F5006F13D0B0F5406FD7
S315080084D014D010214A4A00264FF40040BB422FD13F
S315080084E071B102290FD004290FD0082973D10FE0E2
S315080084F00021EFE70221EDE70421EBE70821E9E790
S31508008500FEF7B0FB03E0104602E0FEF7CFFBE8B348
S31508008510626802EB420181425DD8B0EB023F5AD84D
S31508008520010E03025008181871410023FAF7F4FEE9
S31508008530344AA0F5407191424DD82168C8604BE095
S31508008540E3694FF6EF77834228D1092943D2DFE85A
S3150800855001F005080B420D4242421000FEF782FB6D
S3150800856006E0FEF791FB03E0104602E0FEF79EFBED
S3150800857060B14100606801EB5001B1FBF0F0A0F179
S315080085801001B94227D84FF6F07100E024E0014007
S31508008590C0F3420001432068C1601DE009291AD2D0
S315080085A0DFE801F005080B190D1919191000FEF777
S315080085B059FB06E0FEF768FB03E0104602E0FEF70B
S315080085C075FB48B1616800EB5100B0FBF1F0A0F112
S315080085D01001B94205D90125A6662846E666BDE812
S315080085E0F08180B2A9E7000000800040F369FFEF40
S315080085F00038014000100240004400400048004096
S315080086000024F400FFFC0F0070B54165A0F858205F
S3150800861000210446C0F884102220C4F88000606F48
S31508008620D0B11E4BC362636F1D481863636F1D4844
S315080086305863606F13468163656D21682A46243145
S31508008640606FFDF77FFC38B11020C4F88400202045
S31508008650C4F88000012070BD206940B1216851E846
S31508008660000F40F4807041E80002002AF6D1206825
S31508008670083050E8001F41F0010140E80012002AC6
S31508008680F5D12068083050E8001F41F0400140E865
S315080086900012002AF5D1002070BD0000D182000822
S315080086A0678300088F8200082DE9F0479946174628
S315080086B00D4604464FF00008089E33E0701C31D082
S315080086C0FDF75EFEA0EB0900B04218D8BEB12068DF
S315080086D00168490726D5802D24D0402D22D0C169AE
S315080086E0C94309070DD4082505622046FFF759FE38
S315080086F0C4F8845084F878800120BDE8F087032008
S31508008700FBE7C069C04300050CD421684FF400603C
S3150800871008622046FFF745FE2020C4F8840084F846
S315080087207880ECE72068C06935EA000004D00020AC
S31508008730B842C3D00020E0E70120F9E710B50448A5
S3150800874000F00AFABDE810400148FEF72DBE000009
S31508008750C8000020FEE703B401984100009850EADB
S31508008760C12018BF04204A0D18BF40F0010040F28E
S31508008770FF72B2EB515F08BF40F00200012808BF44
S31508008780052002B070470907090E002804DB00F12E
S31508008790E02080F80014704700F00F0000F1E02098
S315080087A080F8141D704700000FB4802110B503AB84
S315080087B00648029AFAF728FE82B24FF47A730349FA
S315080087C00348FFF70FF810BC5DF814FB980100206A
S315080087D0C800002030380A2801D20120704700203E
S315080087E070470000B5EEC00AF1EE10FA02D89FED08
S315080087F00E0A7047401AB0F5006F02DDA0F58050EA
S3150800880004E010F5006F01DA00F5805000EE900ADA
S315080088109FED061AF8EEE00A20EE811AC1EE000A6C
S31508008820B0EE600A704700000000000000008039C2
S31508008830034610B50020024604E09C5C521C204406
S31508008840C0B2D2B28A42F8D310BD000000B58BB0D0
S3150800885000200121CDE906010390059000900190C2
S3150800886002900891049069460D48FCF73DFF08B14F
S31508008870FCF7BCFD0A48FDF717FA08B1FCF7B6FD88
S3150800888002210748FCF7C0FE08B1FCF7AFFD05203A
S31508008890FDF792FB03A0FFF787FF0BB000BD0000B2
S315080088A04C00002043414E3120696E697469616C41
S315080088B0697A6564207375636365737366756C6C32
S315080088C0790D0A00F0B587B00025CDE90005082026
S315080088D00295CDE903500E468DF814500D4C4FF411
S315080088E07A7709E02068401C2060B84204DD4FF022
S315080088F0FF30256007B0F0BD0748FCF7E7FF002802
S31508008900F0D006AB3246694603482560FCF78EFE72
S315080089100020EFE7300000204C00002007480168DF
S315080089200A6842F010020A600068016841F02001F6
S315080089300160202202490148FEF72EBFC800002028
S31508008940340200202DED028B82B04FF0FF3B9FEDE5
S315080089505C8AFDF7C7FEFFF7B6FAFFF749F9FFF796
S3150800896031F9FFF70DF9FFF789F9FFF7B3F9FFF7C3
S315080089706DFFFFF7D3FFFCF7F5FD0546018851A00B
S31508008980FFF712FFA97856A0FFF70EFFE9785BA05C
S31508008990FFF70AFFDFF88491A978DFF884A189F840
S315080089A00010E9788AF800105E4F07E05E4505D0AA
S315080089B096B1012E51D0022EF8D176E0FCF7D2FC02
S315080089C038B108213846FDF7CDFC6420FDF7F4FAE6
S315080089D0F4E7FCF7B7FC8046012208213846FDF784
S315080089E0C9FCFDF7CDFC0646FCF7ACFC04460A209C
S315080089F0FDF7E2FAFDF7C4FC861B0FD000EE106AFD
S31508008A00B8EE400ADFED480A4146204620EE200A25
S31508008A10FFF7E8FEDFED450A20EE208A99F8000008
S31508008A20A04620B1C8F10000B1EE488A84B29AF88F
S31508008A30000060B118EE100A00F0EEF841EC100BD9
S31508008A40214653EC102B3AA00096FFF7ADFE1021F5
S31508008A503846FDF787FC0126ABE79FED3E0A002165
S31508008A60009128EE000AAA228DF800200191BDEE99
S31508008A70C00A220A8DF8012010EE100A8DF802406D
S31508008A808DF80400020A8DF805108DF806108DF889
S31508008A90032007216846FFF7CBFE8DF807002888D4
S31508008AA06946FFF70FFF28B1022620213846FDF751
S31508008AB059FC7BE7012220213846FDF75BFC8BE752
S31508008AC00000000043757272656E742043414E20A3
S31508008AD049443A203078253032580D0A0000000003
S31508008AE043757272656E7420446972656374696F42
S31508008AF06E3A203078253032580D0A004375727266
S31508008B00656E74204465627567204C6576656C3AB7
S31508008B10203078253032580D0A0000003E0000202B
S31508008B203D000020000400486F12833A0000B44359
S31508008B30416E676C653A2025752C2056656C3A207F
S31508008B40252E32662064743A202575206D730D0A29
S31508008B50000000000000C84210B50446016811482C
S31508008B6081421ED1C869C043C0061AD410200862C3
S31508008B702046FEF7B3FB0C4800684068C0F12000A9
S31508008B80C1B20A4801700A48FFF794FA202108483A
S31508008B90FAF763FD2046BDE8104020220449FEF797
S31508008BA0FBBD10BD00380140500100203C000020EC
S31508008BB03402002010B500290AD00878002807D00A
S31508008BC005487844FBF7B6FF002801D0002010BD01
S31508008BD00248784410BD0000AE020000A60200005C
S31508008BE010B500290AD00878002807D00548784427
S31508008BF0FBF7A0FF002801D0002010BD02487844EA
S31508008C0010BD00009E020000960200000808A0F5AC
S31508008C1000114FEA3101704743004FEAD30C4FEA7F
S31508008C203C0C43401FBF40070CF1605113F0FE4F48
S31508008C3070471CF0006F03D100200CF0004170470C
S31508008C400CF0004343EA507010B540EACC0000F03F
S31508008C500EF800BF000000924FEA0001FFF7D6BFEA
S31508008C604FF000414FF00000A1F5002170470EF1CA
S31508008C70020E2EF0030E5EF8044B244204D44FEA8B
S31508008C804102B2F17F4F11D84FEA4003B3F17F4F4B
S31508008C900CD80ED14FEAD07CB2F17F4F0CEB4C0CBE
S31508008CA00CF1020C08BF4CEBD17C04E04FF0080C29
S31508008CB001E04FEAD17C0CEB4C0324FA03F404F0F0
S31508008CC00704B4F1040C06D20EEB840CBDE8104080
S31508008CD04CF0010C6047DFE80CF0070802024FF081
S31508008CE00040A0F5800010BD0846420018BFD2F12A
S31508008CF0807288BF00F0004010BD4FF04070E1EE72
S31508008D00100A7047FBF772B9FBF7A6BA0000000015
S31508008D10000000000102030406070809A0860100F6
S31508008D20400D0300801A060000350C0040420F0073
S31508008D3080841E0000093D0000127A000024F40019
S31508008D4000366E010048E801006CDC0200000000F5
S31508008D500102030400000000000000003031323335
S31508008D603435363738394142434445464030580051
S31508008D703031323334353637383961626364656683
S31508008D8040307800040000080000000000000002DF
S31508008D900001000010303132333435363738396146
S31508008DA0626364656678700030313233343536373D
S31508008DB038394142434445465850000002400000B5
S31508008DC0000000A00000000005400000000000C8E8
S31508008DD0000000000C4000000000409C000000005D
S31508008DE0194000000020BCBE00000000344000000E
S31508008DF0BFC91B8E00000004B5400000504BCFD001
S31508008E006607E2CF010000006C4100003E8251AACD
S31508008E10DFEEA73401000000D9420000DCB5A0E26D
S31508008E203A301F97FFFFFFFFB4450000FD25A0C895
S31508008E30E9A3C14FFFFFFFFFFF3F000000000080CE
S31508008E4000000000FF3F0000000000800000000056
S31508008E509C8F0008000000204C000000C831000864
S31508008E60E88F00084C0000206C080000E431000878
S31508008E701C00000043000000F8FFFFFF0C00000084
S31508008E800E0000000F0000002E0000001001000078
S31508008E9043000000F8FFFFFF0040404040404040CC
S31508008EA040404141414141404040404040404040AF
S31508008EB04040404040404040400502020202020253
S31508008EC002020202020202020220202020202020A2
S31508008ED020202002020202020202909090909090B6
S31508008EE01010101010101010101010101010101074
S31508008EF010101010020202020202888888888888E8
S31508008F0008080808080808080808080808080808D3
S31508008F1008080808020202024000000000000000DB
S31508008F200000000000000000000000000000000033
S31508008F300000000000000000000000000000000023
S31508008F400000000000000000000000000000000013
S31508008F500000000000000000000000000000000003
S31508008F6000000000000000000000000000000000F3
S31508008F7000000000000000000000000000000000E3
S31508008F8000000000000000000000000000000000D3
S31508008F9000000000000000000000000001000000C2
S31508008FA010000000000000000000000000000000A3
S31508008FB000000000000000000100000000000000A2
S31508008FC0000000000000000000093D00000000004D
S31508008FD00000000000000000000000000000000083
S30D08008FE000000000000000007B
S7050800318D34
